:100000003BC07DC154C053C052C051C050C04FC04E
:100010004EC04DC04CC04BC04AC049C048C047C08C
:1000200046C045C044C00902120001010080190900
:10003000040000000000000012010101FF000008A0
:10004000C016DC050101010200010E03550053003A
:1000500042006100730070001C0377007700770096
:100060002E00660069007300630068006C002E00BB
:10007000640065000403090411241FBECFE5D4E029
:10008000DEBFCDBF10E0A0E6B0E0ECE6FDE002C0D0
:1000900005900D92A236B107D9F710E0A2E6B0E0C4
:1000A00001C01D92A23AB107E1F743D65EC6A8CFC0
:1000B0001F93CF93DF9360919C00662359F16350A7
:1000C00067FD6CC0C2E6D0E0C0919600CF5F20E033
:1000D00010E8809199008D3209F465C08091780014
:1000E00087FD09C0CE0186D52FEF821709F49FC086
:1000F000811120E010E010937800922F209361008E
:1001000010929C009F3F51F486B3837089F1109246
:100110007900E3C0909161009F3FB1F3809160004E
:1001200084FFF2CF692F9930B8F5961B9093610048
:100130001BE48091780080FD13EC8F5F8093780042
:10014000ACE8B0E087FD60C0662309F058C060E00D
:1001500070E0C62F693008F446C02EE18FEF80931F
:10016000610010938B002093600086B3837079F652
:1001700080917900882309F0B0C094E686B383703B
:1001800009F0ABC09150D1F781E080937900909352
:100190009D0090939800A1C068E0C7CF9091610046
:1001A00010929C00AFCF683009F0A5CF888180768F
:1001B00009F056C044E950E02093940089818823D7
:1001C00009F041C02093950022E050939B0040939A
:1001D0009A008F81882309F08ECF8E81821708F0D4
:1001E0008ACF282F88CF8CE890E02CD22C2F2C5F40
:1001F000C83008F0B6CF9FEF90936100B2CFCD0129
:10020000BCD4682F7727A5CFE0919A00F0919B008E
:1002100086FF12C0962F03C084918D933196915022
:10022000D8F7F0939B00E0939A00772792CF8EE166
:100230008093600010E05FCF962F02C081918D9374
:100240009150E0F7EECF8530B9F08630C9F08830B4
:1002500039F1893049F18A3009F0BBCF21E0B5CFBF
:10026000CE01A2D3282F8F3F09F0B3CF888187FF1B
:1002700041CF2E8110E03FCF8A8180939D00A9CF8E
:1002800010EC8B818130A1F08230B1F0833009F025
:10029000A0CF8A818823A1F444E750E024E095CFE1
:1002A0004FE950E021E091CF8A8180939F0091CF68
:1002B00048E350E022E189CF46E250E022E185CFD9
:1002C000813039F0823009F084CF4AE450E02EE0EA
:1002D0007CCF48E550E02CE178CFDF91CF911F91A2
:1002E000089582E690E0809397000B9680939600A5
:1002F00085B7836085BF8BB780648BBF08950F93EC
:100300000FB70F93B09BFECFB09B06C0B09B04C04D
:10031000B09B02C0000000C01F933F932F9331E0B9
:1003200012E006B3102710FD32E0102F3A95C9F7FE
:1003300000FDE3C006B3102720E010FB20F9DF9397
:1003400016B3012700FB21F9CF93C091970006B3A4
:10035000102710FB22F93BE0D0E04F9316B30127A2
:1003600000FB23F94FEF000055C0B09BFECFB09BC0
:1003700006C0B09B04C0B09B02C0000000C0DF916B
:1003800000C0CDCF16B3137079F14F7D206213C03A
:1003900006B3037049F14F7B206415C0037021F14F
:1003A000102F206806B319C006B30370E9F04E7F22
:1003B000216018C039F306B30370B1F0102710FBA9
:1003C00026F9223028F316B3012700FB27F942272C
:1003D00049934FEF06B3243008F3102710FB20F9A0
:1003E000297F11F316B31370E1F1012700FB21F906
:1003F000237FF1F006B30370A1F1102710FB22F95F
:10040000277EE1F016B3012700FB23F93A9541F16D
:100410002F7CD1F006B3037021F1102710FB24F9D3
:100420002F79C1F016B3012700FB25F92F73C2CF36
:1004300016B31370B1F04D7F2260DCCF06B30370AA
:1004400081F04B7F2460DECF16B3137051F0477FED
:100450002860E0CF06B3037021F04F7E2061E2CF29
:100460003BC03C2FC09197003C1B00E433300ABFD7
:1004700098F108811981412F1F77209198000D3242
:1004800079F1013E69F10936C1F00777033421F5AE
:1004900010919E00112301F100919C000030C1F5E4
:1004A0003430C2F130939C00109399000091960073
:1004B000C0939600009397002DC0121769F43091F5
:1004C000600034FD23C00AE500936000CBE8D0E073
:1004D00025C0002700939E004F91CF91DF910DC062
:1004E0001217B9F700939E000AE5009360004F9140
:1004F000CF910AB706FD39CFDF9100E40ABF2F91F3
:100500003F911F910F910FBF0F911895432F03C07B
:100510004AE501C042EDC4E1D0E032E05F9353E030
:10052000C09A08B3B89AB99A20E80FC0052710E01E
:1005300008BB10C0052710E0089408BB13C00527AE
:1005400010E015C0052710E019C020FF052708BBE3
:10055000279517951C3F50F720FF0527279508BBC7
:1005600017951C3F38F720FF05272795179508BBDF
:100570001C3F28F720FF0527279517951C3F08BB30
:1005800008F700C0499120FF052708BB279517955C
:100590001C3F80F520FF0527279508BB17951C3FBA
:1005A00068F520FF05272795179508BB1C3F58F5D0
:1005B00020FF0527279517951C3F08BB38F5242FEA
:1005C0003A9519F60C7F5F9108BB32E03A95F1F746
:1005D00010919D00C651D04011F010939800016019
:1005E00017B31C7F08BB0C7F4F91CF9117BB08BB83
:1005F000DF9183CF052710E008BBCACF052710E0A5
:10060000089408BBCDCF052710E0CFCF052710E019
:10061000D3CFA82FB92F8FEF9FEF41E050EA615061
:1006200070F02D9138E0722F782796958795269552
:1006300070FF02C0842795273A95A9F7F0CF8095DF
:1006400090950895E6DF8D939D930895A398AB9AB6
:10065000000000009B9904C082E58DB91EB8089582
:10066000A29AAA98000000009B9B07C082E58DB962
:1006700081E08EB9A298AA9A089583E58DB91EB833
:10068000A298AA9A0895882339F488E793E0909372
:10069000A1008093A000089585E993E09093A100C4
:1006A0008093A000089592B782B7891B8C30E0F345
:1006B0000895C49AA59AAD9887B38C6287BBC298F7
:1006C000C598F1DFC29AEFDFC2988091A0009091A7
:1006D000A1008559934009F00895B8DF089587B3C4
:1006E000837D87BB88B3837D88BBA5981DB808959B
:1006F0000F931F93CF93C82F00E017E00CC0C3984F
:10070000CC0F000FB4990F5FCEDFC59ACCDFC59830
:10071000115017FD04C0C7FFF2CFC39AF1CF802F4D
:100720009927CF911F910F9108958FB9779BFECF95
:100730008FB1992708951F93CF93CFE103C0C15084
:10074000CF3F51F1E091A000F091A1008CEA099512
:10075000E091A000F091A10083E50995E091A0004F
:10076000F091A10080E00995182FE091A000F09190
:10077000A10080E00995133591F01DB8C59A93DF6B
:10078000C59891DF8091A0009091A1008559934078
:10079000B1F65CDFC150B0F681E090E002C080E0CD
:1007A00090E0CF911F9108950F931F938C0181705A
:1007B000880F880F880FE091A000F091A10080625F
:1007C0000995C801892F99278695E091A000F0919D
:1007D000A100099516950795E091A000F091A10060
:1007E000802F0995E091A000F091A10080E009958B
:1007F00099271F910F9108950F931F93CF93DF9324
:10080000EC01062F142F8170880F880F880FE0915C
:10081000A000F091A10080640995CE01892F99274D
:100820008695E091A000F091A1000995CE019695E2
:100830008795E091A000F091A1000995E091A000BA
:10084000F091A100802F09951123A9F00F3789F0AD
:100850001EE102B7CE01A8DF8F3769F482B7801B93
:100860008D3310F002B711501123A1F781E090E011
:1008700004C08FE08CD080E090E0DF91CF911F9199
:100880000F9108950F931F93CF93DF93EC01162FD1
:10089000E091A000F091A1008CE40995CE01892F90
:1008A00099278695E091A000F091A1000995CE01CD
:1008B00096958795E091A000F091A1000995E091AF
:1008C000A000F091A10080E009951F3F89F01EE192
:1008D00002B7CE0169DF8F3F69F482B7801B8D3389
:1008E00010F002B711501123A1F781E090E004C08D
:1008F0008FE04DD080E090E0DF91CF911F910F917C
:1009000008950F931F938C01E091A000F091A10036
:1009100080EA0995812F9927E091A000F091A1002C
:100920000995E091A000F091A100802F0995E09138
:10093000A000F091A10080E0099599271F910F91E7
:100940000895FF920F931F938C01F62EE091A00063
:10095000F091A10080EC0995812F9927E091A000EA
:10096000F091A1000995E091A000F091A100802FE5
:100970000995E091A000F091A1008F2D09958EE1DD
:1009800006D080E090E01F910F91FF900895382FDE
:1009900020E0231740F492B782B7891B8C33E0F331
:1009A0002F5F2317C0F308951F93CF93DF93EC01BC
:1009B00010E089818130A1F0823009F489C0833050
:1009C00009F489C0843091F0873009F467C085301C
:1009D00009F4C3C0863039F1883009F0C2C09DC027
:1009E0009A9B812F50DE65DEA998BBC08B81992729
:1009F000982F88272A813327822B932B9093860068
:100A0000809385008F819927982F88272E813327FF
:100A1000822B932B90937B0080937A0082E08093CB
:100A20007C001FEF9EC08B819927982F88272A81F1
:100A30003327822B932B90938600809385008C81A3
:100A4000482F552750938800409387002D812F70A1
:100A5000209389008D819927807F9070829592954F
:100A6000907F9827807F9827840F951F9093880008
:100A70008093870020FF04C08091870080938A00C4
:100A80008F819927982F88272E813327822B932BAC
:100A900090937B0080937A0081E0C1CF8B8199276E
:100AA000982F88272A813327822B932B90938600B7
:100AB000809385008F819927982F88272E8133274F
:100AC000822B932B90937B0080937A0083E0A7CFB7
:100AD00006DEA99A46C0E091A000F091A1008A81AB
:100AE000099580937D00E091A000F091A1008B8199
:100AF000099580937E00E091A000F091A1008C8187
:100B0000099580937F00E091A000F091A1008D8174
:100B100009958093800014E024C08B819927982F39
:100B200088272A813327822B932B909386008093EA
:100B300085001092880010928700109389008F81A1
:100B40009927982F88272E813327822B932B9093D8
:100B50007B0080937A0084E062CFEDDD80937D009E
:100B600011E08DE790E090939B0080939A00812F95
:100B70009927DF91CF911F910895EF92FF921F93D4
:100B8000CF937C01162F90917C00892F8250823068
:100B900050F5C0E0C617C0F01FC08091850090914D
:100BA0008600AFDEF701EC0FF11D80838091850098
:100BB0009091860001969093860080938500CF5F88
:100BC000C11750F490917C00923039F780918500E4
:100BD00090918600E9DDE6CF183010F410927C0089
:100BE000812F992702C08FEF90E0CF911F91FF9046
:100BF000EF900895BF92CF92DF92EF92FF920F9302
:100C00001F93CF93DF936C01E62EBB2440917C00B1
:100C1000413019F0443009F080C0FF24FE1408F080
:100C200079C0413009F049C08091870090918800D7
:100C3000892B09F04EC0CF2DDD27FE01EC0DFD1DE7
:100C400060818091850090918600D6DD80917A0048
:100C500090917B00019790937B0080937A00892B81
:100C6000D9F410927C008091890081FF13C080919B
:100C70008A00282F332780918700909188002817B9
:100C8000390741F0CC0DDD1D688180918500909180
:100C90008600F8DDC1E0BC2E809185009091860031
:100CA00001969093860080938500F394FE1490F54E
:100CB00040917C00413009F4B7CFCF2DDD27FE01F4
:100CC000EC0DFD1D6081809185009091860039DEDC
:100CD000BDCFCF2DDD278E010C0D1D1D40E0F8018D
:100CE0006081809185009091860086DD80918A00E8
:100CF000815080938A00882309F0A8CFF801608191
:100D00008091850090918600BDDD80918700809361
:100D10008A009CCF8B2D992702C08FEF90E0DF9146
:100D2000CF911F910F91FF90EF90DF90CF90BF90E8
:100D30000895CFE5D4E0DEBFCDBF12BA18BA8BEF6D
:100D400081BB8FEF87BB90E09150F1F78150D9F7CD
:100D500087BB93E094BB8EEF85BB93BF81E093DCB0
:0C0D6000C0DA7894A5D9A4D9FDCFFFCF4C
:020D6C005AFF2C
:00000001FF
